:020000040000FA
:0400000091EF04F088
:08000800800E016EFE0E06D908
:10001000010E04D9750E0F6E300E8ED1016A018E5D
:100020001D6EFE0EFBD81D50F9D0056A166E176ABC
:1000300000960550D8B40086040E046E173805D813
:10004000175003D8163801D816500F0BF60FD8B03A
:10005000070F0A0F20D0056A166E176A0096055022
:10006000D8B40086050E046E270E136E100E0CD841
:10007000030E136EE80E08D8136A640E05D8136ACF
:100080000A0E02D8165007D0126E17500F6E165077
:100090000E6EACD90E500E6E044E0096055003E065
:1000A000045CD8B007D00E50D8A4009600B602D099
:1000B000300FB4D0120027D80096055003E1008617
:1000C0000A0E056E21C011F020C010F01FC00FF005
:1000D0001EC00EF0046A196A186A176A0A0E166EB4
:1000E00048D9042A0450055CD8A4F5D71650D8A4E2
:1000F000009600A602D0052C03D01650300F8ED8E3
:10010000052EE0D7120021AE1200D880000E1E5638
:100110001F56205621562D0E81D0A66AA68E0900A4
:10012000F55002E002D8FBD712001B6E899A00003E
:100130008998929A92980F0E93161B5000B21ED077
:100140003A0E0F6E980EF8D8330E1A6E28D8130E8A
:100150000F6E880EF1D823D8640EEDD820D8640E27
:10016000EAD8220E1A6E1BD8280E07D80C0E05D816
:10017000060E03D800821B5001D000801A6E00A02A
:1001800009D0899803080AE309D8050E0F6EDC0E22
:10019000D3D812000080FE080FE0898800A00090EC
:1001A000898A0F0E81161A50F00B8112899A1A3A19
:1001B00000B0F5D7640EBFD81B501200ABB2AB989D
:1001C000AB8802C00EF006C00FF0126A136A00007E
:1001D00000D000009EBA13D0E868122613220E2227
:1001E0000F22D8A012001248133CF1D77A0E126EDB
:1001F000136AEFD7ABB2AB98AB889EAAFED7AE50CE
:10020000D8801200A66AA68E0900F55002E002D836
:10021000FBD712009EA8FED7AD6E120001BE85D797
:1002200001B4F8D701A202D001B01ED0008800A806
:10023000009800BA03D0008A35D829E20094080E4D
:10024000136E40D81236132EFCD700B407D000B876
:1002500001D04AD845D841D800B819D843D8D89049
:1002600012501CD0008800A8009800BC05D0FE0BDE
:10027000076E008CD89012D000BE05D01A6E008E8A
:1002800011D805E21A5012D802E200A807D02CD8E3
:1002900027D8009C009E009A009424D81C80D8A0E7
:1002A0001C90120017D8075000BA0109126E080EF0
:1002B000136E123617D801E217D812D80ED8132EA3
:1002C000F8D710D80DD800D00000D89082B8D880C8
:1002D00004D8120007D804D807D8829A949A06D076
:1002E000948A04D0948802D08B9894981200AA6AB9
:1002F000A96EA66AA680A850A94AAA2A1200AA6ACC
:10030000A86EA66AA684550EA76EAA0EA76EA68230
:10031000A6B2FED7A694A94AAA2A1200136A126EA0
:10032000FF0E1226132200D0D8A01200030E0F6E6B
:10033000E30E02D8F5D70F6AF50F0E6EFE0E04E33A
:1003400000D000000E26FDE200000E260F06F9E2A6
:100350000EA002D000D000001200010F036E0A0EA2
:10036000166E176A186A196A04D8032EF8D7165041
:100370001200246A256A266A276A210E146E15D097
:1003800024362536263627361650245C1750255835
:10039000185026581950275808E3276E1650245E27
:1003A0001750255A1850265AD8800E360F36103658
:1003B0001136142EE5D727C019F026C018F025C035
:1003C00017F02450166E1200136A126EF36A080EAC
:1003D000F46E0E36F3361250F35C03E31250F35E04
:1003E000D8801336F42EF5D713501200176A166A08
:1003F000100EF36E0F34163617361250165C13506B
:10040000175805E31250165E1350175AD8800E364F
:100410000F36F32EEFD70E50120011C027F010C088
:1004200026F00FC025F00EC024F026501602F3CFA0
:1004300010F0F4CF11F025501702F3501026F450AD
:10044000112224501802F3501026F4501122275084
:100450001602F350112626501702F350112625508C
:100460001802F350112624501902F350112624507B
:100470001602F3CF0EF0F4CF0FF025501602F35012
:100480000F26F4501022000E112224501702F350B0
:100490000F26F4501022000E112212000E6E11BE13
:1004A00002D80E5012000E1E0F1E101E111E0E2A14
:1004B000D8B00F2AD8B0102AD8B0112A1200E82AD2
:1004C000E806D8B41200D890193218321732163212
:1004D000F7D72020202052462047454E4552415410
:1004E0004F522020202000006279204F4D3342439C
:1004F000202D207665722E20332E3030000046529B
:1005000045513A202020202020202020202020207B
:10051000487A0000202020202020202020202000B9
:1005200020204445425547204D4F44452049532003
:100530004F464620000020204445425547204D4F5D
:100540004445204953204F4E2020000020202020E9
:10055000202020202020202000002020205345544F
:1005600054494E4753204D454E5520202020000031
:1005700052465245513A200045732E53657420204F
:1005800020202020202044776E20557000004469F0
:100590007669646520726174696F202020202020B4
:1005A000202000004D46206F666673657420202071
:1005B0002020202020202020000043616C696272EE
:1005C0006174696F6E2020202020202020200000F0
:1005D000464D207374657073202020202020202039
:1005E000202020200000536E617020746F206772FD
:1005F0006964202020202020202000004D6F6465A9
:1006000020202020202020202020202020202020EA
:10061000000046696C746572202020202020202074
:10062000202020202020000045732E536176652075
:1006300020202020202044776E205570000044693F
:100640007669646520726174696F203D20312020D5
:100650002020000044697669646520726174696FC6
:10066000203D203220202020000044697669646506
:1006700020726174696F203D20342020202000000A
:100680004D46206F6666736574203D203020202023
:100690002020202000004D46206F66667365742080
:1006A0003D2020343535206B487A00004D46206FC0
:1006B0006666736574203D202D343535206B487A8D
:1006C00000004D46206F6666736574203D20313012
:1006D0002E37204D487A00004D46206F66667365C0
:1006E00074203D2D31302E37204D487A00004D4684
:1006F000206F6666736574203D2032312E34204DA4
:10070000487A00004D46206F6666736574203D2D63
:1007100032312E34204D487A00004D46206F6666F7
:10072000736574203D2020637573746F6D20000025
:100730004D46206F6666736574203D202D6375738A
:10074000746F6D2000004E4F4D493A20202020202C
:100750002020202020202020487A00005245414CB3
:100760003A20202020202020202020202020487AED
:1007700000002043616C6962726174696E67207663
:10078000616C75657320000020202020202020202F
:100790002020202020202020202020200000457321
:1007A0002E53617665202020202020204F66662071
:1007B0004F6E0000414D2C20464D206F66667365DC
:1007C00074203D203020487A0000555342206F6647
:1007D00066736574203D202D31353030487A000035
:1007E0004C5342206F6666736574203D202B313573
:1007F0003030487A0000435755206F666673657441
:10080000203D202D38303020487A000043574C20BE
:100810006F6666736574203D202B38303020487A2F
:10082000000046696C7465722069732073657420DA
:1008300020202020202000004672657175656E63BF
:10084000793A20004672657175656E6379206F6E26
:1008500020646973706C61793A2020200000467230
:10086000657175656E6379206F6E20636F6E6E655E
:1008700063746F723A2000004F7574707574206C49
:100880006576656C3A200000537465703A2000006C
:1008900044697669646520726174696F3A2000006A
:1008A0004D46206F66667365743A2000464D20738E
:1008B0007465703A2000536E617020746F20677207
:1008C00069643A2000004D6F64653A200000466973
:1008D0006C7465722073776974636865643A20008C
:1008E000536F6674776172652076657273696F6E97
:1008F00020332E30300020204C4F4144494E4720B9
:1009000044454641554C5420202000002020202002
:1009100020202056414C55455320202020202020C7
:100920000000006A060EAF6E200EAC6E900EAB6E2D
:1009300000010F0E926E936AB70E946EFE0ED36E88
:10094000800E9B6E070EB46ED2980E0ED26E010E04
:10095000C26E0D0EC16EF16AF06AAC98AC84B896A6
:10096000B06A190EAF6E900EAB6E9D6AA16A040E4E
:10097000A06EA26ED08ED288C00EF26E816A9B6B82
:100980009A6B996B010E986F9F6B9E6B9D6B0A0E15
:100990009C6FA36BA26BA16B640EA06FA76BA66B81
:1009A000010EA56FF40EA46FAB6BAA6B030EA96FBB
:1009B000E80EA86FAF6BAE6B040EAD6FE20EAC6FBE
:1009C000B36BB26B090EB16FC40EB06FB76BB66B81
:1009D000130EB56F880EB46FBB6BBA6B180EB96F80
:1009E0006A0EB86FBF6BBE6B200EBD6F8D0EBC6FF5
:1009F000C36BC26B230EC16F280EC06FC76BC66B73
:100A0000270EC56F100EC46FCB6BCA6B300EC96F4B
:100A1000D40EC86FCF6BCE6B610ECD6FA80ECC6FAE
:100A2000D36BD26BC30ED16F500ED06FD76B010E4C
:100A3000D66F860ED56FA00ED46FDB6B020EDA6F09
:100A4000490ED96FF00ED86FDF6B030EDE6F0D0EFF
:100A5000DD6F400EDC6FE36B070EE26FA10EE16FFE
:100A6000200EE06FE76B0F0EE66F420EE56F400E53
:100A7000E46FEB6B980EEA6F960EE96F800EE86FED
:100A8000EF6BEE6BED6B010EEC6FF36BF26BF16BDA
:100A90000A0EF06FF76BF66BF56B640EF46FFB6B81
:100AA000FA6B030EF96FE80EF86FFF6BFE6B270E03
:100AB000FD6F100EFC6F0101036B010E026F860EBD
:100AC000016FA00E006F076B0F0E066F420E056FD1
:100AD000400E046F0B6B980E0A6F960E096F800E16
:100AE000086F000104EC00F0800E016E0EEC00F0C7
:100AF000040EF76ED20EF66E8DEC00F0800E016ED5
:100B0000C00E0EEC00F0040EF76EE80EF66E8DECE3
:100B100000F0C80E8B6F96918D6B886B586A8E6B48
:100B20009693969D506A4F6A4E6A4D6A546A536A0C
:100B3000526A516A956B010EAA6E0E0EA96E79EC7F
:100B400001F0356E79EC01F0366E79EC01F0376E1C
:100B500079EC01F0386E010EAA6E150EA96E79ECD3
:100B600001F0396E79EC01F03A6E79EC01F03B6EF0
:100B700079EC01F03C6E010EAA6E140EA96E79ECB0
:100B800001F08F6F010EAA6E1E0EA96E79EC01F0B6
:100B9000926F968992A19699968B96A9969B010E33
:100BA000AA6E130EA96E79EC01F0926F92C094F0C8
:100BB000010EAA6E120EA96E79EC01F0916F91C030
:100BC00093F09651E8B814D0D8909235E96EEA6A5D
:100BD000EA36E936EA36EC0EE926000EEA22EFCFD5
:100BE0002DF0ECCF2EF0ECCF2FF0ECCF30F013D077
:100BF000D8909135E96EEA6AEA36E936EA36980E17
:100C0000E926000EEA22EFCF2DF0ECCF2EF0ECCF4C
:100C10002FF0ECCF30F0010EAA6E1F0EA96E79EC0A
:100C200001F0806F978180A19791010EAA6E190E35
:100C3000A96E79EC01F0806F38C044F037C043F002
:100C400036C042F035C041F08F5107E0D8904136B0
:100C5000423643364436E82EF9D7000E445C0EE3A4
:100C60000BE12D0E435C0AE307E12A0E425C06E32A
:100C700003E1800E415C02E3000E01D0010E286EFC
:100C8000410E415C8E0E4258530E4358380E445864
:100C9000000102E2000E01D0010E281212E0030E44
:100CA000196E5B0E186E600E176E166A8F515FEC30
:100CB00002F019C038F018C037F017C036F016C06F
:100CC00035F058EC0DF00B0E136EB80E8FEC01F0F2
:100CD000800E016E0EEC00F0040EF76EFE0EF66E46
:100CE0008DEC00F0320E866FA6EC13F058EC0DF090
:100CF0007EEC14F0BAEC11F080A4FED741D1715013
:100D00005D6E70505C6E6F505B6E6E505A6E596ABD
:100D10007550616E7450606E73505F6E72505E6E8F
:100D2000636A646A656A666A440E7C6E59365A362E
:100D30005B365C365D3663366436653666366150E2
:100D4000665CD8A4B0EF06F06050655CD8A4B0EF44
:100D500006F05F50645CD8A4B0EF06F05E50635CB0
:100D6000D8A0C3EF06F05E50635E5F50D8A05F3C32
:100D7000645E6050D8A0603C655E6150D8A0613C64
:100D8000665ED8905980D8907C2E96EF06F01200BF
:100D90007FEC06F05D50776E5C50786E5B50796E3C
:100DA0005A507A6E59507B6E240E855DD8A0DFEFC5
:100DB00006F0D8907732783279327A327B327D6A97
:100DC0008351766E84517C6E7D6AD8907C327D3200
:100DD0007C327D327C5076127D5077121200676A29
:100DE000666A656A646A636A5D6A59505E02F3CF37
:100DF00063F0F4CF64F05A505E02F3506426E86A60
:100E0000F420656E5B505E02F3506526E86AF420BC
:100E1000666E5C505E02F3506626E86AF420676EE8
:100E200012006C505D6E6B505C6E6A505B6E695068
:100E30005A6E6850596E5F6A6D505E6E636A646A7E
:100E4000280E7C6E59365A365B365C365D36633614
:100E500064365F50645CD8A430EF07F05E50635C8A
:100E6000D8A03DEF07F05E50D8A05E3C635E5F50B7
:100E7000D8A05F3C645ED8905980D8907C2E22EF39
:100E800007F01200D8905D325C325B325A32593230
:100E90005C50756E5B50746E5A50736E5950726E22
:100EA0001200D89059365A365B365C365D36D8908B
:100EB00059365A365B365C365D36D89059365A36D6
:100EC0005B365C365D36D89059365A365B365C36C2
:100ED0005D36636A646A656A666A676A480E7C6E34
:100EE00059365A365B365C365D366336643665365F
:100EF000663667366250675CD8A490EF07F06150A1
:100F0000665CD8A490EF07F06050655CD8A490EFC1
:100F100007F05F50645CD8A490EF07F05E50635C0C
:100F2000D8A0A7EF07F05E50635E5F50D8A05F3C8B
:100F3000645E6050D8A0603C655E6150D8A0613CA2
:100F4000665E6250D8A0623C675ED8905980D890A7
:100F50007C2E70EF07F06D505E6EEFEC06F0675080
:100F60006C6E66506B6E65506A6E6450696E63504D
:100F7000686ED890683669366A366B366C36120001
:100F8000066A0A0E026EDEEC00F003E3886F59EF8A
:100F90001FF082B09ED0320E8EEC01F082B099D05C
:100FA0009651E8B81BD092C094F0922B080E925D37
:100FB000D8B0926BD8909235E96EEA6AEA36E93693
:100FC000EA36EC0EE926000EEA22EFCF2DF0ECCF48
:100FD0002EF0ECCF2FF0ECCF30F01BD091C093F07F
:100FE000912B150E915D02E3140E916FD8909135FF
:100FF000E96EEA6AEA36E936EA36980EE926000E24
:10100000EA22EFCF2DF0ECCF2EF0ECCF2FF0ECCF8B
:1010100030F096310BE3800E016EC00E0EEC00F046
:10102000050EF76E140EF66E8DEC00F0BAEC11F0B2
:101030008C6B82B04ED08C2B050E8EEC01F0C90E5D
:101040008C5DD8A045D09691800E016EC00E0EEC3E
:1010500000F0050EF76E200EF66E8DEC00F0030E1C
:10106000136EE80E8FEC01F09651E8B816D094C0DC
:1010700092F0D8909235E96EEA6AEA36E936EA36B5
:10108000EC0EE926000EEA22EFCF2DF0ECCF2EF089
:10109000ECCF2FF0ECCF30F015D093C091F0D8907A
:1010A0009135E96EEA6AEA36E936EA36980EE926BB
:1010B000000EEA22EFCF2DF0ECCF2EF0ECCF2FF088
:1010C000ECCF30F07EEC14F0BAEC11F082A0FED739
:1010D000B0D784B695D0320E8EEC01F084B690D0A5
:1010E0009651E8B81CD092C094F09207650E925DBC
:1010F00002E3070E926FD8909235E96EEA6AEA36FB
:10110000E936EA36EC0EE926000EEA22EFCF2DF0A2
:10111000ECCF2EF0ECCF2FF0ECCF30F01BD091C005
:1011200093F09107650E915D02E3140E916FD890D4
:101130009135E96EEA6AEA36E936EA36980EE9262A
:10114000000EEA22EFCF2DF0ECCF2EF0ECCF2FF0F7
:10115000ECCF30F096310BE3800E016EC00E0EEC3A
:1011600000F0050EF76E140EF66E8DEC00F0BAEC82
:1011700011F08C6B84B644D08C2B050E8EEC01F0F4
:10118000C90E8C5D3CE39681800E016EC00E0EECA4
:1011900000F0050EF76E360EF66E8DEC00F09651EF
:1011A000E8B816D094C092F0D8909235E96EEA6A09
:1011B000EA36E936EA36EC0EE926000EEA22EFCFEF
:1011C0002DF0ECCF2EF0ECCF2FF0ECCF30F015D08F
:1011D00093C091F0D8909135E96EEA6AEA36E93623
:1011E000EA36980EE926000EEA22EFCF2DF0ECCF7A
:1011F0002EF0ECCF2FF0ECCF30F084A6FED7BAD78C
:1012000082B2EDD0320E8EEC01F091C093F082B23A
:10121000E1D0196A2D0E186E2A0E176E800E166E0A
:101220008F515FEC02F019C044F018C043F017C0B2
:1012300042F016C041F030C034F02FC033F02EC061
:1012400032F02DC031F09651E8B82ED04150355CC7
:101250000A6E425036580B6E435037580C6E44504D
:1012600038580D6E31500A5C32500B5833500C58C0
:1012700034500D5818E234C011F033C010F032C0B1
:101280000FF031C00EF0196A186A176A0A0E166E4E
:10129000B9EC01F011C034F010C033F00FC032F0DF
:1012A0000EC031F0D3D72ED04150355C0A6E42507B
:1012B00036580B6E435037580C6E445038580D6EEC
:1012C00031500A5C32500B5833500C5834500D5882
:1012D00019E29153D8A49107D8909135E96EEA6A42
:1012E000EA36E936EA36980EE926000EEA22EFCF12
:1012F00031F0ECCF32F0ECCF33F0ECCF34F091534F
:10130000D8A4D2D73150355E3250365A3350375A7E
:101310003450385A4150355C425036584350375853
:101320004450385808E244C038F043C037F042C057
:1013300036F041C035F02F5030101BE12D508D0A92
:1013400018E12E50200A15E138C011F037C010F016
:1013500036C00FF035C00EF0000EADEC01F00A6E95
:10136000070E0A5C05E13506000E365A375A385A20
:1013700025D09651E8AC22D038C011F037C010F01B
:1013800036C00FF035C00EF034C019F033C018F07D
:1013900032C017F031C016F0B9EC01F027C044F0AC
:1013A00026C043F025C042F024C041F04150355ED4
:1013B0004250365A4350375A4450385AA6EC13F02C
:1013C000F3D91F0E8B5D02E30A0E8B5F8B518EECFF
:1013D00001F01DD793C091F0C80E8B6F968382B435
:1013E0008CD0320E8EEC01F082B484D02D50352694
:1013F0002E5036222F5037223050382238C00DF070
:1014000037C00CF036C00BF035C00AF08F5107E042
:10141000D8900A360B360C360D36E82EF9D7410E29
:101420000A5C8E0E0B58530E0C58380E0D5813E3F1
:10143000380E196E530E186E8E0E176E400E166E05
:101440008F515FEC02F019C038F018C037F017C0A8
:1014500036F016C035F02F5030101BE12D508D0A9C
:1014600018E12E50200A15E138C011F037C010F0F5
:1014700036C00FF035C00EF0000EADEC01F00A6E74
:10148000090E0A5C05E1352A000E36223722382281
:1014900025D09651E8AC22D038C011F037C010F0FA
:1014A00036C00FF035C00EF030C019F02FC018F064
:1014B0002EC017F02DC016F0B9EC01F027C044F093
:1014C00026C043F025C042F024C041F04150355EB3
:1014D0004250365A4350375A4450385AA6EC13F00B
:1014E00063D91F0E8B5D02E30A0E8B5F8B518EEC6E
:1014F00001F07AD7C80E8B6F968380B625D1320E55
:101500008EEC01F080B620D180C082F08053D8A448
:1015100080077EEC14F08C6B80B616D18C2B050EF8
:101520008EEC01F0C90E8C5DD8A00DD19691800E85
:10153000016E0EEC00F0460E95EC00F04D0E95ECB1
:1015400000F0530E95EC00F03A0E95EC00F0965139
:10155000E8A80AD06F0E95EC00F06E0E95EC00F046
:10156000200E95EC00F008D06F0E95EC00F0660EA2
:1015700095EC00F095EC00F0800E016E870E0EECFD
:1015800000F0200E95EC00F0530E95EC00F0740E78
:1015900095EC00F0670E95EC00F03A0E95EC00F03B
:1015A0009651E8AC0AD06F0E95EC00F06E0E95ECFB
:1015B00000F0200E95EC00F008D06F0E95EC00F0D6
:1015C000660E95EC00F095EC00F08F5303E1010EF0
:1015D000906F03D0D8908F35906F800E016E8F0E74
:1015E0000EEC00F0200E95EC00F0440E95EC00F0AF
:1015F000520E95EC00F03A0E95EC00F0010E056EDF
:1016000090512CEC00F0800E016EC00E0EEC00F03C
:101610004F0E95EC00F0660E95EC00F095EC00F0A6
:10162000730E95EC00F03A0E95EC00F0056A3CC0A4
:1016300021F03BC020F03AC01FF039C01EF05BEC37
:1016400000F0050EF76E4C0EF66E8DEC00F0800E7D
:10165000016ECF0E0EEC00F04D0E95EC00F03A0E40
:1016600095EC00F0545053105210511009E1460E01
:1016700095EC00F04D0E95EC00F0200E95EC00F08E
:101680005150240A12E15250FA0A0FE15350FF0A56
:101690000CE15450FF0A09E1550E95EC00F0530E91
:1016A00095EC00F0420E95EC00F0535054100FE111
:1016B0005150DC0A0CE15250050A09E14C0E95EC40
:1016C00000F0530E95EC00F0420E95EC00F05150F6
:1016D000E00A12E15250FC0A0FE15350FF0A0CE1FC
:1016E0005450FF0A09E1430E95EC00F0570E95ECBB
:1016F00000F0550E95EC00F0535054100FE151508E
:10170000200A0CE15250030A09E1430E95EC00F067
:10171000570E95EC00F04C0E95EC00F0070E136E92
:10172000D00E8FEC01F080A6FED782C080F0800E34
:10173000016E0EEC00F0040EF76EFE0EF66E8DECF0
:1017400000F068EF06F0E8D680B42CD0320E8EECB4
:1017500001F080B427D080C082F00B0E805DD8A04D
:10176000802B7EEC14F08C6B80B41CD08C2B050E7F
:101770008EEC01F0C90E8C5D14E3969182C080F06E
:1017800080A64DEF25F0800E016E0EEC00F0050EE8
:10179000F76E5A0EF66E8DEC00F042EF15F080A455
:1017A000FED7E2D7C0EF07F039503524296E3A5002
:1017B00036202A6E3B5037202B6E3C5038202C6E42
:1017C000515029241E6E52502A201F6E53502B2038
:1017D000206E54502C20216E21C02CF020C02BF004
:1017E0001FC02AF01EC029F08F5107E0D89029367B
:1017F0002A362B362C36E82EF9D711DA29C06EF0AE
:101800002AC06FF02BC070F02CC071F08551865D3E
:10181000D8B446D08551040DF3CF1EF0F4CF1FF09D
:101820001FC08AF01EC089F08AC0AAFF89C0A9FF24
:1018300079EC01F0756E010E8925A96E000E8A21E2
:10184000AA6E79EC01F0746E020E8925A96E000E65
:101850008A21AA6E79EC01F0736E030E8925A96EB8
:10186000000E8A21AA6E79EC01F0726E8A6BAC0EC2
:10187000896F85518925A96E000E8A21AA6E79EC9F
:1018800001F0846F8A6BD70E896F85518925A96E07
:10189000000E8A21AA6E79EC01F0836F85C086F074
:1018A000C8EC06F029504D5C0E6E2A504E580F6E53
:1018B0002B504F58106E2C505058116E4FEC02F0B8
:1018C0001E6E0FC01FF010C020F011C021F021C00B
:1018D00011F020C010F01FC00FF01EC00EF0196AEA
:1018E000186A030E176EE80E166E0DEC02F011C0AA
:1018F00044F010C043F00FC042F00EC041F050C0A1
:1019000011F04FC010F04EC00FF04DC00EF0196A2C
:10191000186A030E176EE80E166EB9EC01F011C0CE
:1019200021F010C020F00FC01FF00EC01EF044C008
:1019300011F043C010F042C00FF041C00EF021C0C2
:1019400019F020C018F01FC017F01EC016F0B9EC37
:1019500001F011C00DF010C00CF00FC00BF00EC064
:101960000AF00C500D1007E1E50E0A5C0C0E0B5846
:1019700002E2000E01D0010E286E000E96B3010E99
:1019800028123DE0AA0E34EC01F0890E34EC01F08F
:10199000100E32EC01F0AA0E34EC01F0070E34EC1C
:1019A00001F0765034EC01F0775034EC01F07850CF
:1019B00034EC01F0795034EC01F07A5034EC01F061
:1019C0007B5032EC01F0AA0E34EC01F0890E34ECBD
:1019D00001F0000E32EC01F0AA0E34EC01F0870E9B
:1019E00034EC01F0400E32EC01F02CC050F02BC072
:1019F0004FF02AC04EF029C04DF096932AD0AA0E7F
:101A000034EC01F0870E34EC01F0200E32EC01F0E2
:101A1000AA0E34EC01F0070E34EC01F0765034ECF1
:101A200001F0775034EC01F0785034EC01F079504B
:101A300034EC01F07A5034EC01F07B5032EC01F0E0
:101A4000AA0E34EC01F0870E34EC01F0000E32ECFB
:101A500001F09631D8A01200800E016EC00E0EEC7F
:101A600000F0050EF76E700EF66E8DEC00F0240E91
:101A70000EEC01F0020E056E765016EC00F0020E30
:101A8000056E775016EC00F0020E056E785016ECDD
:101A900000F0020E056E795016EC00F0020E056E95
:101AA0007A5016EC00F0020E056E7B5016EF00F037
:101AB00039503524296E3A5036202A6E3B50372053
:101AC0002B6E3C5038202C6E515029241E6E5250E3
:101AD0002A201F6E53502B20206E54502C20216E34
:101AE00021C02CF020C02BF01FC02AF01EC029F00E
:101AF0008F5107E0D89029362A362B362C36E82E1F
:101B0000F9D78DD829C06EF02AC06FF02BC070F0C5
:101B10002CC071F08551040DF3CF1EF0F4CF1FF0EF
:101B20001FC08AF01EC089F08AC0AAFF89C0A9FF21
:101B300079EC01F0756E010E8925A96E000E8A21DF
:101B4000AA6E79EC01F0746E020E8925A96E000E62
:101B50008A21AA6E79EC01F0736E030E8925A96EB5
:101B6000000E8A21AA6E79EC01F0726E8A6BAC0EBF
:101B7000896F85518925A96E000E8A21AA6E79EC9C
:101B800001F0846F8A6BD70E896F85518925A96E04
:101B9000000E8A21AA6E79EC01F0836F85C086F071
:101BA000C8EC06F0AA0E34EC01F0890E34EC01F01A
:101BB000100E32EC01F0AA0E34EC01F0070E34ECFA
:101BC00001F0765034EC01F0775034EC01F07850AD
:101BD00034EC01F0795034EC01F07A5034EC01F03F
:101BE0007B5032EC01F0AA0E34EC01F0890E34EC9B
:101BF00001F0000E32EC01F0AA0E34EC01F0870E79
:101C000034EC01F0400E32EC01F02CC050F02BC04F
:101C10004FF02AC04EF029C04DF096931200070EE7
:101C2000876F9731D8A04DD0410E295C4B0E2A58B2
:101C30004C0E2B58000E2C5802E3010E876F810EBC
:101C4000295C960E2A58980E2B58000E2C5802E349
:101C5000020E876F010E295C2D0E2A58310E2B586B
:101C6000010E2C5802E3030E876F010E295C5A0EF9
:101C70002A58620E2B58020E2C5802E3040E876F6E
:101C8000010E295CB40E2A58C40E2B58040E2C5891
:101C900002E3050E876F010E295C680E2A58890E33
:101CA0002B58090E2C5802E3060E876F010E295C93
:101CB000D00E2A58120E2B58130E2C5802E3070E82
:101CC000876F87B1808E87A1809E87B3808C87A322
:101CD000809C87B5828687A58296410E295C8E0EF0
:101CE0002A58530E2B58380E2C580BE3380E2C6EF6
:101CF000530E2B6E8E0E2A6E400E296E2A0E856FA5
:101D00001200300E2C5C10E30BE1470E2B5C0CE351
:101D100007E19E0E2A5C08E303E1800E295C04E3E0
:101D20002A0E0001856F1200290E2C5C10E30BE1D6
:101D3000B90E2B5C0CE307E1270E2A5C08E303E1F4
:101D4000000E295C04E3290E0001856F1200240EA9
:101D50002C5C10E30BE15B0E2B5C0CE307E1DC0E6B
:101D60002A5C08E303E1800E295C04E3280E0001ED
:101D7000856F1200200E2C5C10E30BE1C80E2B5C6B
:101D80000CE307E1550E2A5C08E303E1800E295CB1
:101D900004E3270E0001856F12001D0E2C5C10E37A
:101DA0000BE1CD0E2B5C0CE307E1650E2A5C08E32A
:101DB00003E1000E295C04E3260E0001856F12008A
:101DC0001A0E2C5C10E30BE1D20E2B5C0CE307E146
:101DD000740E2A5C08E303E1800E295C04E3250EFF
:101DE0000001856F1200180E2C5C10E30BE1230E2E
:101DF0002B5C0CE307E1CF0E2A5C08E303E1400E05
:101E0000295C04E3240E0001856F1200140E2C5C83
:101E100010E30BE1DC0E2B5C0CE307E1930E2A5C74
:101E200008E303E1800E295C04E3230E0001856FC3
:101E30001200120E2C5C10E30BE17A0E2B5C0CE30B
:101E400007E1390E2A5C08E303E1800E295C04E314
:101E5000220E0001856F1200100E2C5C10E30BE1C6
:101E6000170E2B5C0CE307E1DF0E2A5C08E303E1AD
:101E7000800E295C04E3210E0001856F12000E0E16
:101E80002C5C10E30BE19A0E2B5C0CE307E1670E70
:101E90002A5C08E303E1400E295C04E3200E000104
:101EA000856F12000D0E2C5C10E30BE13B0E2B5CDA
:101EB0000CE307E1730E2A5C08E303E1800E295C62
:101EC00004E31F0E0001856F12000C0E2C5C10E362
:101ED0000BE1110E2B5C0CE307E1E70E2A5C08E333
:101EE00003E1A00E295C04E31E0E0001856F1200C1
:101EF0000A0E2C5C10E30BE15F0E2B5C0CE307E198
:101F0000070E2A5C08E303E1800E295C04E31D0E42
:101F10000001856F1200090E2C5C10E30BE10F0E1F
:101F20002B5C0CE307E1560E2A5C08E303E1000E8C
:101F3000295C04E31C0E0001856F1200080E2C5C66
:101F400010E30BE10B0E2B5C0CE307E1EF0E2A5CB8
:101F500008E303E1C00E295C04E31B0E0001856F5A
:101F60001200070E2C5C10E30BE1540E2B5C0CE30B
:101F700007E1D40E2A5C08E303E1C00E295C04E308
:101F80001A0E0001856F1200060E2C5C10E30BE1A7
:101F90009D0E2B5C0CE307E1B90E2A5C08E303E11C
:101FA000C00E295C04E3190E0001856F1200050EB6
:101FB0002C5C10E30BE1D70E2B5C0CE307E15C0E0D
:101FC0002A5C08E303E1800E295C04E3180E00019B
:101FD000856F1200050E2C5C10E30BE12F0E2B5CBD
:101FE0000CE307E1830E2A5C08E303E1C00E295CE1
:101FF00004E3170E0001856F1200040E2C5C10E341
:102000000BE1870E2B5C0CE307E1AB0E2A5C08E3C7
:1020100003E1000E295C04E3160E0001856F120037
:10202000040E2C5C10E30BE1050E2B5C0CE307E1C6
:10203000F70E2A5C08E303E1E00E295C04E3150EC9
:102040000001856F1200030E2C5C10E30BE1750E8E
:102050002B5C0CE307E1020E2A5C08E303E1800E2F
:10206000295C04E3140E0001856F1200030E2C5C42
:1020700010E30BE1190E2B5C0CE307E1750E2A5CF3
:1020800008E303E1000E295C04E3130E0001856FF1
:102090001200020E2C5C10E30BE1AE0E2B5C0CE385
:1020A00007E1A50E2A5C08E303E1400E295C04E386
:1020B000120E0001856F1200020E2C5C10E30BE182
:1020C000530E2B5C0CE307E1170E2A5C08E303E1D7
:1020D000C00E295C04E3110E0001856F1200020E90
:1020E0002C5C10E30BE1020E2B5C0CE307E1380ED5
:1020F0002A5C08E303E1A00E295C04E3100E000152
:10210000856F1200010E2C5C10E30BE1BA0E2B5C04
:102110000CE307E1810E2A5C08E303E1400E295C31
:1021200004E30F0E0001856F1200010E2C5C10E31A
:102130000BE1860E2B5C0CE307E1A00E2A5C08E3A2
:1021400003E1000E295C04E30E0E0001856F12000E
:10215000010E2C5C10E30BE1570E2B5C0CE307E146
:10216000520E2A5C08E303E1A00E295C04E30D0E85
:102170000001856F1200010E2C5C10E30BE12B0EA9
:102180002B5C0CE307E1120E2A5C08E303E1800EEE
:10219000295C04E30C0E0001856F1200010E2C5C1B
:1021A00010E30BE1040E2B5C0CE307E1EC0E2A5C60
:1021B00008E303E1E00E295C04E30B0E0001856FE8
:1021C0001200000E2C5C10E30BE1E00E2B5C0CE324
:1021D00007E14D0E2A5C08E303E1E00E295C04E30D
:1021E0000A0E0001856F1200000E2C5C10E30BE15B
:1021F000C10E2B5C0CE307E1C90E2A5C08E303E186
:10220000600E295C04E3090E0001856F1200000EC8
:102210002C5C10E30BE1A70E2B5C0CE307E1D80E5E
:102220002A5C08E303E1C00E295C04E3080E000108
:10223000856F1200000E2C5C10E30BE1900E2B5CFE
:102240000CE307E1F50E2A5C08E303E1600E295C6C
:1022500004E3070E0001856F1200000E2C5C10E3F2
:102260000BE17D0E2B5C0CE307E11F0E2A5C08E3FB
:1022700003E1400E295C04E3060E0001856F1200A5
:10228000000E2C5C10E30BE16C0E2B5C0CE307E101
:10229000560E2A5C08E303E1600E295C04E3050E98
:1022A0000001856F1200000E2C5C10E30BE15D0E47
:1022B0002B5C0CE307E1140E2A5C08E303E1200E1B
:1022C000295C04E3040E0001856F1200000E2C5CF3
:1022D00010E30BE1500E2B5C0CE307E1DF0E2A5CF0
:1022E00008E303E1200E295C04E3030E0001856F7F
:1022F0001200000E2C5C10E30BE1460E2B5C0CE38D
:1023000007E1300E2A5C08E303E1C00E295C04E318
:10231000020E0001856F1200000E2C5C10E30BE131
:102320003D0E2B5C0CE307E1090E2A5C08E303E198
:10233000000E295C04E3010E0001856F1200000EFF
:102340002C5C0FE30BE12D0E2B5C0BE307E12A0E57
:102350002A5C07E303E1800E295C03E30001856B3F
:102360001200856B2C6A2D0E2B6E2A0E2A6E800EA3
:10237000296E1200800E016ECB0E0EEC00F0530E93
:1023800095EC00F0740E95EC00F0650E95EC00F005
:10239000700E95EC00F03A0E95EC00F02D042E1026
:1023A0002F1030100BE1200E95EC00F095EC00F0B2
:1023B000310E95EC00F0200E95EF00F02D500A0A3A
:1023C0002E102F1030100CE1200E95EC00F0310E85
:1023D00095EC00F0300E95EC00F0200E95EF00F03B
:1023E0002D50640A2E102F1030100BE1310E95EC99
:1023F00000F0300E95EC00F095EC00F0200E95EF1B
:1024000000F02F50301012E12D50E80A0FE12E504D
:10241000030A0CE1310E95EC00F02E0E95EC00F065
:10242000300E95EC00F06B0E95EF00F02F50301051
:1024300012E12D50100A0FE12E50270A0CE1200E58
:1024400095EC00F0310E95EC00F0300E95EC00F0BC
:102450006B0E95EF00F02D50A00A13E12E50860A66
:1024600010E12F50010A0DE130520BE1310E95ECD5
:1024700000F0300E95EC00F095EC00F06B0E95EF4F
:1024800000F02D50400A13E12E50420A10E12F5067
:102490000F0A0DE130520BE1200E95EC00F095ECA7
:1024A00000F0310E95EC00F04D0E95EF00F02D5040
:1024B000800A14E12E50960A11E12F50980A0EE17D
:1024C00030520CE1200E95EC00F0310E95EC00F04E
:1024D000300E95EC00F04D0E95EF00F02F503010BF
:1024E00011E12D50F40A0EE12E50010A0BE1350ED8
:1024F00095EC00F0300E95EC00F095EC00F0200E1D
:1025000095EF00F02D50400A13E12E500D0A10E116
:102510002F50030A0DE130520BE1320E95EC00F022
:10252000300E95EC00F095EC00F06B0E95EF00F09E
:102530002D50200A13E12E50A10A10E12F50070A56
:102540000DE130520BE1350E95EC00F0300E95ECBC
:1025500000F095EC00F06B0E95EF00F02F5030106E
:1025600012E12D50C40A0FE12E50090A0CE1320E7F
:1025700095EC00F02E0E95EC00F0350E95EC00F089
:102580006B0E95EF00F02F50301012E12D50880A9D
:102590000FE12E50130A0CE1350E95EC00F02E0ED3
:1025A00095EC00F0300E95EC00F06B0E95EF00F01E
:1025B0002F50301012E12D50280A0FE12E50230A1F
:1025C0000CE1390E95EC00F02E0E95EC00F0300E7B
:1025D00095EC00F06B0E95EF00F02F50301012E1EB
:1025E0002D50A80A0FE12E50610A0CE1200E95EC47
:1025F00000F0320E95EC00F0350E95EC00F06B0E0D
:1026000095EF00F02F50301012E12D50500A0FE1DD
:102610002E50C30A0CE1200E95EC00F0350E95EC1F
:1026200000F0300E95EC00F06B0E95EF00F02D50A1
:10263000F00A14E12E50490A11E12F50020A0EE16E
:1026400030520CE1310E95EC00F0350E95EC00F0B7
:10265000300E95EC00F06B0E95EF00F0800E016EE1
:10266000CB0E0EEC00F0530E95EC00F0740E95ECD2
:1026700000F03A0E95EC00F0200E95EC00F02F5093
:10268000301015E12D50D40A12E12E50300A0FE11E
:10269000310E95EC00F0320E95EC00F02E0E95EC1C
:1026A00000F0350E95EC00F06B0E95EF00F02F501A
:1026B000301015E12D50E20A12E12E50040A0FE10C
:1026C000310E95EC00F02E0E95EC00F0320E95ECEC
:1026D00000F0350E95EC00F06B0E95EF00F02F50EA
:1026E000301015E12D506A0A12E12E50180A0FE140
:1026F000360E95EC00F02E0E95EC00F0320E95ECB7
:1027000000F0350E95EC00F06B0E95EF00F02F50B9
:10271000301014E12D508D0A11E12E50200A0EE1E7
:10272000380E95EC00F02E0E95EC00F0330E95EC83
:1027300000F095EC00F06B0E95EF00F0306A2F6A18
:102740002E6A640E2D6E969915D61200800E016EBB
:10275000850E0EEC00F0200E95EC00F0000E355CBE
:10276000E10E3658F50E3758050E385803E2200EA4
:1027700095EC00F0800E355C960E3658980E375862
:10278000000E385803E2200E95EC00F0800E016E2A
:10279000056A38C011F037C010F036C00FF035C0F0
:1027A0000EF0196A0F0E186E420E176E400E166E5E
:1027B000B9EC01F011C021F010C020F00FC01FF0E3
:1027C0000EC01EF05CEC00F02E0E95EC00F0030E37
:1027D000056E38C011F037C010F036C00FF035C0AC
:1027E0000EF0196A186A030E176EE80E166EB9EC31
:1027F00001F011C021F010C020F00FC01FF00EC07A
:102800001EF05CEC00F02E0E95EC00F0030E056E51
:1028100038C021F037C020F036C01FF035C01EF0A0
:102820005CEF00F0800E016EC50E0EEC00F0200E85
:1028300095EC00F0000E295CE10E2A58F50E2B589D
:10284000050E2C5803E2200E95EC00F0800E295C5A
:10285000960E2A58980E2B58000E2C5803E2200E84
:1028600095EC00F0800E016E056A2CC011F02BC0B3
:1028700010F02AC00FF029C00EF0196A0F0E186E62
:10288000420E176E400E166EB9EC01F011C021F029
:1028900010C020F00FC01FF00EC01EF05CEC00F066
:1028A0002E0E95EC00F0030E056E2CC011F02BC01F
:1028B00010F02AC00FF029C00EF0196A186A030E32
:1028C000176EE80E166EB9EC01F011C021F010C0C1
:1028D00020F00FC01FF00EC01EF05CEC00F02E0EBA
:1028E00095EC00F0030E056E2CC021F02BC020F0FB
:1028F0002AC01FF029C01EF05CEF00F09631D8B05E
:102900001200800E016EC00E0EEC00F04F0E95EC22
:1029100000F0550E95EC00F0540E95EC00F03A0ED8
:1029200095EC00F080C081F080530AE1200E95EC18
:1029300000F0310E95EC00F0300E95EC00F094D0E4
:10294000010E805D09E1200E95EC00F095EC00F0A1
:10295000350E95EC00F088D0020E805D09E1200E66
:1029600095EC00F095EC00F0300E95EC00F07CD08A
:10297000030E805D0AE1200E95EC00F02D0E95EC23
:1029800000F0350E95EC00F06FD0040E805D0AE18A
:102990002D0E95EC00F0310E95EC00F0300E95EC1C
:1029A00000F062D0050E805D0AE12D0E95EC00F07E
:1029B000310E95EC00F0350E95EC00F055D0060E7A
:1029C000805D0AE12D0E95EC00F0320E95EC00F0E2
:1029D000300E95EC00F048D0070E805D0AE12D0E18
:1029E00095EC00F0320E95EC00F0350E95EC00F011
:1029F0003BD0080E805D0CE10C0E816F2D0E95EC26
:102A000000F0330E95EC00F0300E95EC00F02CD079
:102A1000090E805D0CE10D0E816F2D0E95EC00F01E
:102A2000330E95EC00F0350E95EC00F01DD00A0E3B
:102A3000805D0CE10E0E816F2D0E95EC00F0340ED2
:102A400095EC00F0300E95EC00F00ED00B0E805D92
:102A50000BE12D0E95EC00F0340E95EC00F0350EE8
:102A600095EC00F00F0E816F81C081FF640E95EC34
:102A700000F0420E95EC00F06D0E95EC00F0200E8B
:102A800095EF00F0800E016EC00E0EEC00F0050E0A
:102A9000F76E780EF66E8DEC00F08D530BE1800E24
:102AA000016E0EEC00F0050EF76E8E0EF66E8DECDC
:102AB00000F053D0010E8D5D0BE1800E016E0EEC27
:102AC00000F0050EF76EA40EF66E8DEC00F045D00A
:102AD000020E8D5D0BE1800E016E0EEC00F0050E16
:102AE000F76EBA0EF66E8DEC00F037D0030E8D5DEA
:102AF0000BE1800E016E0EEC00F0050EF76ED00EAD
:102B0000F66E8DEC00F029D0040E8D5D0BE1800E89
:102B1000016E0EEC00F0050EF76EE60EF66E8DEC13
:102B200000F01BD0050E8D5D0BE1800E016E0EECEA
:102B300000F0050EF76EFC0EF66E8DEC00F00DD079
:102B4000060E8D5D0AE1800E016E0EEC00F0060EA1
:102B5000F76E120EF66E8DEC00F080A6FED780A404
:102B6000FED782A2FED782A4FED782B40AD0320E4C
:102B70008EEC01F082A48D2B070E8D5DD8B08D6B8D
:102B800081D782B20BD0320E8EEC01F082A28D077B
:102B9000650E8D5D02E3060E8D6F74D780B623D06F
:102BA000320E8EEC01F080B61ED08D510E6E0608EE
:102BB0001AE3FA6AD8900E36FA360E36FA36CA0E8C
:102BC0000E262B0EFA220E50F96EFFEF15F06AEF6B
:102BD00016F023EF19F06FEF1BF0ABEF1CF0D9EFFD
:102BE0001DF0CCEF1EF080B409D0320E8EEC01F057
:102BF00080B404D082C080F068EF06F0B6D7800EB3
:102C0000016EC00E0EEC00F0060EF76E280EF66E8A
:102C10008DEC00F08F530BE1800E016E0EEC00F096
:102C2000060EF76E3E0EF66E8DEC00F01BD0010E18
:102C30008F5D0BE1800E016E0EEC00F0060EF76E5C
:102C4000540EF66E8DEC00F00DD0020E8F5D0AE191
:102C5000800E016E0EEC00F0060EF76E6A0EF66E38
:102C60008DEC00F080A4FED780A6FED782A2FED70E
:102C700082A4FED782B40AD0320E8EEC01F082A478
:102C80008F2B030E8F5DD8B08F6BB9D782B20BD06C
:102C9000320E8EEC01F082A28F07650E8F5D02E38B
:102CA000020E8F6FACD780B60DD0320E8EEC01F0D5
:102CB00080B608D0010EAA6E140EA96E8F5180EC5A
:102CC00001F0E0D680B405D0320E8EEC01F080A485
:102CD000D9D6D0D73C503B103A10391002E1586A8F
:102CE00062D03950580A0BE13A50F10A08E13B50E2
:102CF000060A05E13C5203E1010E586E54D03950EA
:102D0000A80A0CE13A500E0A09E13B50F90A06E123
:102D10003C50FF0A03E1020E586E45D03950E00ADC
:102D20000BE13A50440A08E13B50A30A05E13C524A
:102D300003E1030E586E37D03950200A0CE13A50A7
:102D4000BB0A09E13B505C0A06E13C50FF0A03E183
:102D5000040E586E28D03950C00A0CE13A50890A46
:102D600009E13B50460A06E13C50010A03E1050E29
:102D7000586E19D03950400A0CE13A50760A09E1F0
:102D80003B50B90A06E13C50FE0A03E1060E586EBC
:102D90000AD039503A103B103C1003E0070E586E31
:102DA00002D0080E586E800E016EC00E0EEC00F0C0
:102DB000060EF76E280EF66E8DEC00F058520FE1FD
:102DC000800E016E0EEC00F0060EF76E800EF66EB1
:102DD0008DEC00F04C6A4B6A4A6A496AA3D0010E36
:102DE000585C12E1800E016E0EEC00F0060EF76EDC
:102DF000960EF66E8DEC00F04C6A060E4B6EF10EE0
:102E00004A6E580E496E8ED0020E585C12E1800E4A
:102E1000016E0EEC00F0060EF76EAC0EF66E8DEC49
:102E200000F04C68F90E4B6E0E0E4A6EA80E496EFD
:102E300079D0030E585C12E1800E016E0EEC00F0AA
:102E4000060EF76EC20EF66E8DEC00F04C6AA30E05
:102E50004B6E440E4A6EE00E496E64D0040E585C10
:102E600012E1800E016E0EEC00F0060EF76ED80E29
:102E7000F66E8DEC00F04C685C0E4B6EBB0E4A6E2D
:102E8000200E496E4FD0050E585C13E1800E016E86
:102E90000EEC00F0060EF76EEE0EF66E8DEC00F006
:102EA000010E4C6E460E4B6E890E4A6EC00E496E78
:102EB00039D0060E585C13E1800E016E0EEC00F066
:102EC000070EF76E040EF66E8DEC00F0FE0E4C6EE3
:102ED000B90E4B6E760E4A6E400E496E23D0070E29
:102EE000585C0FE1800E016E0EEC00F0070EF76EDD
:102EF0001A0EF66E8DEC00F04C6A4B6A4A6A496A0B
:102F000011D0080E585C0EE1800E016E0EEC00F040
:102F1000070EF76E300EF66E8DEC00F04C6A4B6AC1
:102F20004A6A496A80A4FED780A6FED782A2FED74D
:102F300082A4FED782B40AD0320E8EEC01F082A4B5
:102F4000582A090E585CD8B0586A2DD782B20BD0D7
:102F5000320E8EEC01F082A25806650E585C02E338
:102F6000080E586E20D780B624D0320E8EEC01F0B9
:102F700080B61FD0070E585C1BE24CC03CF04BC023
:102F80003BF04AC03AF049C039F0010EAA6E150E66
:102F9000A96E395080EC01F03A5080EC01F03B50C2
:102FA00080EC01F03C5080EC01F042EF15F001D0D4
:102FB00009D080B406D0320E8EEC01F080A442EF2E
:102FC00015F0B8D738C044F037C043F036C042F0EF
:102FD00035C041F03CC011F03BC010F03AC00FF0DA
:102FE00039504EEC02F0356E0FC036F010C037F09D
:102FF00011C038F030C034F02FC033F02EC032F0A2
:103000002DC031F0306A2F6A030E2E6EE80E2D6E41
:10301000800E016E0EEC00F0040EF76EFE0EF66EE2
:103020008DEC00F080A4FED780A6FED782A2FED74A
:1030300082A4FED7A6EC13F082B220D0320E8EEC22
:1030400001F082B219D02D50355E2E50365A2F50D5
:10305000375A3050385A38AE04D0386A376A366A30
:10306000356AA6EC13F01F0E8B5D02E30A0E8B5F30
:103070008B518EEC01F0E5D7C80E8B6F82B41AD05D
:10308000320E8EEC01F082B413D02D5035262E5026
:1030900036222F50372230503822A6EC13F01F0E64
:1030A0008B5D02E30A0E8B5F8B518EEC01F0EBD748
:1030B000C80E8B6F82B036D0320E8EEC01F082B02B
:1030C00031D0800E016ECA0E0EEC00F0200E95EC91
:1030D00000F030C011F02FC010F02EC00FF02DC046
:1030E0000EF0196A186A176A0A0E166E0DEC02F0D5
:1030F00011C030F010C02FF00FC02EF00EC02DF018
:10310000810E2D5C960E2E58980E2F58000E3058BA
:1031100005E3306A2F6A2E6A010E2D6EBAEC11F0AB
:1031200082A0FED784B634D0320E8EEC01F084B685
:103130002FD0800E016ECA0E0EEC00F0200E95EC22
:1031400000F030C011F02FC010F02EC00FF02DC0D5
:103150000EF0196A186A176A0A0E166EB9EC01F0B9
:1031600011C030F010C02FF00FC02EF00EC02DF0A7
:1031700030502F102E102D1007E1306A980E2F6E50
:10318000960E2E6E800E2D6EBAEC11F084A6FED730
:1031900080B63FD0320E8EEC01F080B63AD0070EEA
:1031A000585C09E138C03CF037C03BF036C03AF01B
:1031B00035C039F00CD035500008396E000E365449
:1031C0003A6E000E37543B6E000E38543C6E44C0CD
:1031D00038F043C037F042C036F041C035F0010E40
:1031E000AA6E150EA96E395080EC01F03A5080ECB1
:1031F00001F03B5080EC01F03C5080EC01F034C019
:1032000030F033C02FF032C02EF031C02DF042EF3D
:1032100015F080B417D0320E8EEC01F080B412D0CD
:1032200044C038F043C037F042C036F041C035F0FA
:1032300034C030F033C02FF032C02EF031C02DF04A
:1032400042EF15F0F9D680A6FED730C034F02FC07B
:1032500033F02EC032F02DC031F0306A2F6A2E6A62
:103260000A0E2D6E8FC090F08F6B38C044F037C0BF
:1032700043F036C042F035C041F02CC038F02BC0CE
:1032800037F02AC036F029C035F0800E016E0EEC02
:1032900000F0070EF76E460EF66E8DEC00F0A6EC11
:1032A00013F0800E016EC00E0EEC00F0070EF76EEC
:1032B0005C0EF66E8DEC00F012EC14F080A4FED7DC
:1032C00080A6FED782A2FED782A4FED782B04BD0C2
:1032D000320E8EEC01F082B046D030C011F02FC01B
:1032E00010F02EC00FF02DC00EF0196A186A176A80
:1032F0000A0E166E0DEC02F011C030F010C02FF067
:103300000FC02EF00EC02DF0810E2D5C960E2E58A3
:10331000980E2F58000E305805E3306A2F6A2E6A37
:10332000010E2D6E800E016EC00E0EEC00F0050E2B
:10333000F76E140EF66E8DEC00F0BAEC11F0010E83
:10334000136EF40E8FEC01F082A0FED7800E016E9A
:10335000C00E0EEC00F0070EF76E5C0EF66E8DECF4
:1033600000F012EC14F084B649D0320E8EEC01F06D
:1033700084B644D030C011F02FC010F02EC00FF032
:103380002DC00EF0196A186A176A0A0E166EB9EC8B
:1033900001F011C030F010C02FF00FC02EF00EC0A1
:1033A0002DF030502F102E102D1007E1306A980E9E
:1033B0002F6E960E2E6E800E2D6E800E016EC00E3C
:1033C0000EEC00F0050EF76E140EF66E8DEC00F0AC
:1033D000BAEC11F0010E136EF40E8FEC01F084A61E
:1033E000FED7800E016EC00E0EEC00F0070EF76ED9
:1033F0005C0EF66E8DEC00F012EC14F082B21AD076
:10340000320E8EEC01F082B213D02D50295E2E5078
:103410002A5A2F502B5A30502C5A12EC14F01F0EEF
:103420008B5D02E30A0E8B5F8B518EEC01F0EBD7C4
:10343000C80E8B6F82B41AD0320E8EEC01F082B4BB
:1034400013D02D5029262E502A222F502B223050B7
:103450002C2212EC14F01F0E8B5D02E30A0E8B5F20
:103460008B518EEC01F0EBD7C80E8B6F80B61AD063
:10347000320E8EEC01F080B615D030D844C038F052
:1034800043C037F042C036F041C035F034C030F0B0
:1034900033C02FF032C02EF031C02DF090C08FF02D
:1034A00042EF15F080B419D0320E8EEC01F080B4EA
:1034B00014D044C038F043C037F042C036F041C0A9
:1034C00035F034C030F033C02FF032C02EF031C0B0
:1034D0002DF090C08FF042EF15F0F8D6800E016EFF
:1034E0000EEC00F0070EF76E720EF66E8DEC00F02B
:1034F000800E016EC00E0EEC00F0070EF76E880E07
:10350000F66E8DEC00F00FEC0EF0AA0E34EC01F02C
:10351000070E34EC01F018EC01F07C6E18EC01F0B1
:10352000626E18EC01F0616E18EC01F0606E18EC40
:1035300001F05F6E16EC01F05E6E7C38E842070B1E
:103540007D6ED8907C347F6ED8907F367F8262AE5D
:103550007F927F8062AC7F907F9E7F2A3F0E6216B3
:10356000010EAA6E020E7D24A96ED8B0AA2A79ECAB
:1035700001F07E6E7E507F02F4CF56F0F3CF55F00F
:10358000563055306D6E29C059F02AC05AF02BC004
:103590005BF02CC05CF05D6A51EC07F0856B2B0E84
:1035A000855DD8B097D0AA6AD70E8525A96ED8B008
:1035B000AA2A79EC01F07E6E7E38E842070B7E6E17
:1035C000010EAA6E020E7E24A96ED8B0AA2A79EC4A
:1035D00001F06D6E11EC07F0AA6AAC0E8525A96E9C
:1035E000D8B0AA2A79EC01F06D6E6D2A5F6A6DC0C1
:1035F0005EF01EEC07F0240E855D03E248EC07F058
:1036000002D042EC07F08551040DF3CF1EF0F4CF49
:103610001FF01FC0AAFF1EC0A9FF755080EC01F06B
:103620001F6A1E6A236A040E226E23C00EF08551A3
:103630002202F3CF22F0F4CF23F00E02F350232620
:1036400022501E2623501F22010E1E24A96E000E9A
:103650001F20AA6E745080EC01F01F6A1E6A236A54
:10366000040E226E23C00EF085512202F3CF22F009
:10367000F4CF23F00E02F350232622501E262350AF
:103680001F22020E1E24A96E000E1F20AA6E735068
:1036900080EC01F01F6A1E6A236A040E226E23C0AA
:1036A0000EF085512202F3CF22F0F4CF23F00E0268
:1036B000F350232622501E2623501F22030E1E24C1
:1036C000A96E000E1F20AA6E725080EC01F0852BAF
:1036D000D8A065D7010E136EF40E8FEF01F092C0E3
:1036E00094F091C093F0800E016E0EEC00F0050E88
:1036F000F76ED00EF66E8DEC00F0800E016EC00EEF
:103700000EEC00F0070EF76E9E0EF66E8DEC00F0DC
:10371000968B96A9969B80A4FED780A6FED782A200
:10372000FED782A4FED79651E8A80FD0800E016E76
:10373000890E0EEC00F06F0E95EC00F06E0E95EC1D
:1037400000F0200E95EC00F00DD0800E016E890E79
:103750000EEC00F06F0E95EC00F0660E95EC00F0AC
:1037600095EC00F082B416D0320E8EEC01F082B4EB
:1037700011D09689800E016E890E0EEC00F06F0E4E
:1037800095EC00F06E0E95EC00F0200E95EC00F03C
:1037900082A4FED782B215D0320E8EEC01F082B236
:1037A00010D09699800E016E890E0EEC00F06F0E0F
:1037B00095EC00F0660E95EC00F095EC00F082A21E
:1037C000FED780B668D0320E8EEC01F080B663D0A2
:1037D00093C091F094C092F09651E8A81BD0D89075
:1037E0009135E96EEA6AEA36E936EA36980EE92654
:1037F000000EEA22EFCF2DF0ECCF2EF0ECCF2FF021
:10380000ECCF30F0010EAA6E1E0EA96E010E80ECF8
:1038100001F01AD0D8909235E96EEA6AEA36E936B4
:10382000EA36EC0EE926000EEA22EFCF2DF0ECCFBF
:103830002EF0ECCF2FF0ECCF30F0010EAA6E1E0E62
:10384000A96E000E80EC01F09651E8AC22D038C091
:1038500011F037C010F036C00FF035C00EF030C098
:1038600019F02FC018F02EC017F02DC016F0B9ECCB
:1038700001F027C044F026C043F025C042F024C028
:1038800041F04150355E4250365A4350375A445009
:10389000385A42EF15F080B45DD0320E8EEC01F054
:1038A00080B458D0968996AB969993C091F093C006
:1038B00092F09651E8A814D0D8909135E96EEA6A52
:1038C000EA36E936EA36980EE926000EEA22EFCF0C
:1038D0002DF0ECCF2EF0ECCF2FF0ECCF30F013D05A
:1038E000D8909235E96EEA6AEA36E936EA36EC0EA5
:1038F000E926000EEA22EFCF2DF0ECCF2EF0ECCF30
:103900002FF0ECCF30F09651E8AC22D038C011F057
:1039100037C010F036C00FF035C00EF030C019F0CF
:103920002FC018F02EC017F02DC016F0B9EC01F022
:1039300027C044F026C043F025C042F024C041F027
:103940004150355E4250365A4350375A4450385AE7
:1039500042EF15F007D792C094F091C093F0968F84
:1039600096AD969F800E016E0EEC00F0050EF76E80
:10397000E60EF66E8DEC00F0800E016EC00E0EECC1
:1039800000F0070EF76E9E0EF66E8DEC00F080A430
:10399000FED780A6FED782A2FED782A4FED796517C
:1039A000E8AC0FD0800E016E8D0E0EEC00F06F0EA5
:1039B00095EC00F06E0E95EC00F0200E95EC00F00A
:1039C0000DD0800E016E8D0E0EEC00F06F0E95EC9A
:1039D00000F0660E95EC00F095EC00F082B416D085
:1039E000320E8EEC01F082B411D0968D800E016EF5
:1039F0008D0E0EEC00F06F0E95EC00F06E0E95EC57
:103A000000F0200E95EC00F082A4FED782B215D013
:103A1000320E8EEC01F082B210D0969D800E016EB7
:103A20008D0E0EEC00F06F0E95EC00F0660E95EC2E
:103A300000F095EC00F082A2FED780B65AD0320E8C
:103A40008EEC01F080B655D09651E8A816D093C000
:103A500091F0D8909135E96EEA6AEA36E936EA36AD
:103A6000980EE926000EEA22EFCF2DF0ECCF2EF0D3
:103A7000ECCF2FF0ECCF30F015D094C092F0D8906E
:103A80009235E96EEA6AEA36E936EA36EC0EE9265C
:103A9000000EEA22EFCF2DF0ECCF2EF0ECCF2FF07E
:103AA000ECCF30F09651E8AC22D038C011F037C0DE
:103AB00010F036C00FF035C00EF030C019F02FC036
:103AC00018F02EC017F02DC016F0B9EC01F027C089
:103AD00044F026C043F025C042F024C041F04150DC
:103AE000355E4250365A4350375A4450385A42EFA6
:103AF00015F080B45DD0320E8EEC01F080B458D059
:103B0000968996AB96999651E8A816D093C091F0F5
:103B1000D8909135E96EEA6AEA36E936EA36980EC7
:103B2000E926000EEA22EFCF2DF0ECCF2EF0ECCFFD
:103B30002FF0ECCF30F015D094C092F0D8909235A1
:103B4000E96EEA6AEA36E936EA36EC0EE926000E54
:103B5000EA22EFCF2DF0ECCF2EF0ECCF2FF0ECCF10
:103B600030F09651E8AC22D038C011F037C010F0D8
:103B700036C00FF035C00EF030C019F02FC018F06D
:103B80002EC017F02DC016F0B9EC01F027C044F09C
:103B900026C043F025C042F024C041F04150355EBC
:103BA0004250365A4350375A4450385A42EF15F073
:103BB00015D7545053105210511002E1956B41D05B
:103BC0005150240A0CE15250FA0A09E15350FF0AFD
:103BD00006E15450FF0A03E1010E956F32D05350B5
:103BE000541009E15150DC0A06E15250050A03E184
:103BF000020E956F26D05150E00A0CE15250FC0A9B
:103C000009E15350FF0A06E15450FF0A03E1030E95
:103C1000956F17D05350541009E15150200A06E116
:103C20005250030A03E1040E956F0BD0800E016E13
:103C3000C00E0EEC00F0060EF76E280EF66E8DEC40
:103C400000F095530FE1800E016E0EEC00F0070EB0
:103C5000F76EB40EF66E8DEC00F04C6A4B6A4A6A51
:103C6000496A4FD0010E955D11E1800E016E0EEC98
:103C700000F0070EF76ECA0EF66E8DEC00F04C6881
:103C80004B68FA0E4A6E240E496E3BD0020E955DCB
:103C900011E1800E016E0EEC00F0070EF76EE00EE3
:103CA000F66E8DEC00F04C6A4B6A050E4A6EDC0E27
:103CB000496E27D0030E955D11E1800E016E0EEC6A
:103CC00000F0070EF76EF60EF66E8DEC00F04C6805
:103CD0004B68FC0E4A6EE00E496E13D0040E955DE3
:103CE00010E1800E016E0EEC00F0080EF76E0C0E67
:103CF000F66E8DEC00F04C6A4B6A030E4A6E200E95
:103D0000496E80A4FED780A6FED782A2FED782A4E9
:103D1000FED782B40AD0320E8EEC01F082A4952B2D
:103D2000050E955DD8B0956B8CD782B20BD0320E54
:103D30008EEC01F082A29507650E955D02E3040EFC
:103D4000956F7FD780B61FD0320E8EEC01F080B613
:103D50001AD04CC054F04BC053F04AC052F049C086
:103D600051F0010EAA6E1A0EA96E515080EC01F0AE
:103D7000525080EC01F0535080EC01F0545080EC34
:103D800001F042EF15F080B406D0320E8EEC01F057
:103D900080A442EF15F0BDD7800E016E0EEC00F04E
:103DA000080EF76E220EF66E8DEC00F0800E016E9E
:103DB000C00E0EEC00F0070EF76E9E0EF66E8DEC48
:103DC00000F080A4FED780A6FED782A2FED782A4F0
:103DD000FED797310FE3800E016E8E0E0EEC00F0D1
:103DE0006F0E95EC00F06E0E95EC00F0200E95EC49
:103DF00000F00DD0800E016E8E0E0EEC00F06F0EF6
:103E000095EC00F0660E95EC00F095EC00F082B4B5
:103E100016D0320E8EEC01F082B411D09781800E54
:103E2000016E8E0E0EEC00F06F0E95EC00F06E0E33
:103E300095EC00F0200E95EC00F082A4FED782B243
:103E400015D0320E8EEC01F082B210D09791800E18
:103E5000016E8E0E0EEC00F06F0E95EC00F0660E0B
:103E600095EC00F095EC00F082A2FED780B618D059
:103E7000320E8EEC01F080B613D0973108E3010EBC
:103E8000AA6E1F0EA96E010E80EC01F007D0010E84
:103E9000AA6E1F0EA96E000E80EC01F042EF15F025
:103EA00080B406D0320E8EEC01F080A442EF15F003
:103EB000AED7610E885D000ED8B0010E286E7B0E65
:103EC000885D02E3000E01D0010E2816D8A4889B5D
:103ED000460E885DD8A45BD0446A436A426A416A50
:103EE000130E066E880E026EDEEC00F0D8A040EFD6
:103EF00025F0886F0D0E885D25E1800E415C2A0E4D
:103F000042582D0E4358000E445802E2000E01D0D4
:103F1000010E286E410E415C8E0E4258530E4358DE
:103F2000380E445802E3000E01D0010E28160AE0B4
:103F300044C038F043C037F042C036F041C035F0DD
:103F400040EF25F044C011F043C010F042C00FF024
:103F500041C00EF0196A186A176A0A0E166E0DEC47
:103F600002F011C044F010C043F00FC042F00EC088
:103F700041F088510F0B216A206A1F6A1E6E41268C
:103F80001F5042222050432221504422A9D7530ED1
:103F9000885DD8A4E2D0346A336A326A316A130E7B
:103FA000066E880E026EDEEC00F0D8A040EF25F021
:103FB000886F4B0E885D010ED8A4000E286E6B0E24
:103FC000885D010ED8A4000E2812D8B447D0130E75
:103FD000066E880E026EDEEC00F0D8A040EF25F0F1
:103FE000886F0D0E885D36E13104321033103410C5
:103FF00002E0000E01D0010E286E31500A0A321084
:104000003310341002E0000E01D0010E281231509E
:10401000640A32103310341002E0000E01D0010E99
:10402000281218E034C011F033C010F032C00FF085
:1040300031C00EF0196A186A030E176EE80E166E7C
:104040000DEC02F011C030F010C02FF00FC02EF0B8
:104050000EC02DF0BAEC11F040EF25F04D0E885D4A
:10406000010ED8A4000E286E6D0E885D010ED8A436
:10407000000E28123EE0130E066E880E026EDEEC75
:1040800000F0D8A040EF25F0886F0D0E885D2DE17F
:10409000310432103310341002E0000E01D0010E52
:1040A000286E31500A0A32103310341002E0000E2C
:1040B00001D0010E281219E034C011F033C010F005
:1040C00032C00FF031C00EF0196A0F0E186E420E9A
:1040D000176E400E166E0DEC02F011C030F010C0DD
:1040E0002FF00FC02EF00EC02DF0BAEC11F040EF03
:1040F00025F00D0E885D0CE134C030F033C02FF098
:1041000032C02EF031C02DF0BAEC11F040EF25F0A6
:1041100034C011F033C010F032C00FF031C00EF0D7
:10412000196A186A176A0A0E166E0DEC02F011C0B1
:1041300034F010C033F00FC032F00EC031F08851AF
:104140000F0B216A206A1F6A1E6E31261F50322211
:10415000205033222150342222D74C0E885DD8A41F
:10416000AED0576A130E066E880E026EDEEC00F0BB
:10417000D8A040EF25F0886F2D0E885D49E0350E00
:10418000885D11E1130E066E880E026EDEEC00F003
:10419000D8A040EF25F0886F0D0E885D02E1010E7A
:1041A000806F40EF25F0310E885D1DE1130E066E25
:1041B000880E026EDEEC00F0D8A040EF25F0886F8C
:1041C000300E885D10E1130E066E880E026EDEEC76
:1041D00000F0D8A040EF25F0886F0D0E885DD8B4B0
:1041E000806B40EF25F0300E885D11E1130E066EF6
:1041F000880E026EDEEC00F0D8A040EF25F0886F4C
:104200000D0E885D02E1020E806F40EF25F057D061
:10421000130E066E880E026EDEEC00F0D8A040EFA2
:1042200025F0886F0F0E8815576E350E885D31E0CA
:10423000130E066E880E026EDEEC00F0D8A040EF82
:1042400025F0886F0D0E885D0CE157C00EF0050E4D
:10425000E4EC01F0576E020E5724806F40EF25F01A
:1042600018D01F6A0A0E1E6E1FC00EF057501E0295
:10427000F3CF1EF0F4CF1FF00E02F3501F26236A77
:1042800088C022F00F0E2216000E23161E50222484
:10429000576E130E066E880E026EDEEC00F0D8A08C
:1042A00040EF25F0886F0D0E885D09E157C00EF0D4
:1042B000050EE4EC01F0576E020E5724806F520E8B
:1042C000885DD8A4E2EF23F0130E066E880E026E0E
:1042D000DEEC00F0D8A040EF25F0886F0D0E885D71
:1042E000D8A470D20D0E0AEC01F00A0E0AEC01F00F
:1042F000040EF76ED20EF66E02EC01F00D0E0AEC13
:1043000001F00A0E0AEC01F038C044F037C043F067
:1043100036C042F035C041F08F5309E1080EF76E08
:10432000380EF66E02EC01F089EC25F021D0080E73
:10433000F76E440EF66E02EC01F089EC25F038C001
:1043400044F037C043F036C042F035C041F08F51E1
:1043500007E0D8904136423643364436E82EF9D746
:10436000080EF76E5E0EF66E02EC01F089EC25F099
:10437000080EF76E780EF66E02EC01F0805307E13E
:10438000310E0AEC01F0300E0AEC01F07FD0010E84
:10439000805D04E1350E0AEC01F078D0020E805DFC
:1043A00004E1300E0AEC01F071D0030E805D07E1EC
:1043B0002D0E0AEC01F0350E0AEC01F067D0040E68
:1043C000805D0AE12D0E0AEC01F0310E0AEC01F0DD
:1043D000300E0AEC01F05AD0050E805D0AE12D0E78
:1043E0000AEC01F0310E0AEC01F0350E0AEC01F096
:1043F0004DD0060E805D0AE12D0E0AEC01F0320E62
:104400000AEC01F0300E0AEC01F040D0070E805D9E
:104410000AE12D0E0AEC01F0320E0AEC01F0350E25
:104420000AEC01F033D0080E805D0AE12D0E0AEC93
:1044300001F0330E0AEC01F0300E0AEC01F026D048
:10444000090E805D0AE12D0E0AEC01F0330E0AEC34
:1044500001F0350E0AEC01F019D00A0E805D0AE178
:104460002D0E0AEC01F0340E0AEC01F0300E0AECCD
:1044700001F00CD00B0E805D09E12D0E0AEC01F06D
:10448000340E0AEC01F0350E0AEC01F0200E0AECB5
:1044900001F0640E0AEC01F0420E0AEC01F06D0E20
:1044A0000AEC01F00D0E0AEC01F00A0E0AEC01F024
:1044B000080EF76E880EF66E02EC01F0305218E12D
:1044C0002F5016E1E80E2D5C030E2E5811E2040E5B
:1044D000016E056A30C021F02FC020F02EC01FF001
:1044E0002DC01EF05CEC00F0200E0AEC01F051D063
:1044F000400E2D5C420E2E580F0E2F58000E3058D5
:1045000024E2040E016E056A30C011F02FC010F0D5
:104510002EC00FF02DC00EF0196A186A030E176E28
:10452000E80E166EB9EC01F011C021F010C020F0B9
:104530000FC01FF00EC01EF05CEC00F0200E0AEC65
:1045400001F06B0E0AEC01F024D0040E016E056A36
:1045500030C011F02FC010F02EC00FF02DC00EF0A3
:10456000196A0F0E186E420E176E400E166EB9ECD9
:1045700001F011C021F010C020F00FC01FF00EC0DC
:104580001EF05CEC00F0200E0AEC01F04D0E0AEC7F
:1045900001F0D8908F35886F8853D8B4882B480E97
:1045A0000AEC01F07A0E0AEC01F00D0E0AEC01F0B3
:1045B0000A0E0AEC01F0080EF76E900EF66E02EC91
:1045C00001F0040E016E88512BEC00F00D0E0AEC88
:1045D00001F00A0E0AEC01F0080EF76EA00EF66E5E
:1045E00002EC01F0040E016E056A3CC021F03BC0F4
:1045F00020F03AC01FF039C01EF05BEC00F0200E36
:104600000AEC01F0480E0AEC01F07A0E0AEC01F017
:104610000D0E0AEC01F00A0E0AEC01F0080EF76E1E
:10462000AC0EF66E02EC01F09651E8A807D06F0EC2
:104630000AEC01F06E0E0AEC01F008D06F0E0AECE5
:1046400001F0660E0AEC01F00AEC01F00D0E0AEC26
:1046500001F00A0E0AEC01F0080EF76EB60EF66EC7
:1046600002EC01F09651E8AC07D06F0E0AEC01F0B5
:104670006E0E0AEC01F008D06F0E0AEC01F0660E27
:104680000AEC01F00AEC01F00D0E0AEC01F00A0E42
:104690000AEC01F0080EF76EC60EF66E02EC01F0A1
:1046A00054505310521051100FE1410E0AEC01F01A
:1046B0004D0E0AEC01F02C0E0AEC01F0460E0AEC4D
:1046C00001F04D0E0AEC01F05150240A12E1525053
:1046D000FA0A0FE15350FF0A0CE15450FF0A09E1B6
:1046E000550E0AEC01F0530E0AEC01F0420E0AECF2
:1046F00001F0535054100FE15150DC0A0CE15250BC
:10470000050A09E14C0E0AEC01F0530E0AEC01F027
:10471000420E0AEC01F05150E00A12E15250FC0A3C
:104720000FE15350FF0A0CE15450FF0A09E1430E18
:104730000AEC01F0570E0AEC01F0550E0AEC01F0FC
:10474000535054100FE15150200A0CE15250030A0B
:1047500009E1430E0AEC01F0570E0AEC01F04C0E91
:104760000AEC01F00D0E0AEC01F00A0E0AEC01F061
:10477000080EF76ECE0EF66E02EC01F09651E8AC24
:1047800007D06F0E0AEC01F06E0E0AEC01F008D0B3
:104790006F0E0AEC01F0660E0AEC01F00AEC01F073
:1047A0000D0E0AEC01F00A0E0AEC01F0080EF76E8D
:1047B000E00EF66E02EC01F00D0E0AEC01F00A0EAE
:1047C0000AEC01F0440E885D1EE1130E066E880EA1
:1047D000026EDEEC00F0D8A053D1886F070E88156A
:1047E0001F6A1E6E1F301E30906F130E066E880EED
:1047F000026EDEEC00F0D8A043D1886F0D0E885D0C
:1048000002E190C08FF04F0E885DD8A45DD0406A61
:104810003F6A3E6A3D6A9697130E066E880E026ED8
:10482000DEEC00F0D8A02CD1886F2D0E885D02E15F
:104830009687F2D70D0E885D22E140C03CF03FC064
:104840003BF03EC03AF03DC039F09651E8A616D094
:104850003CC011F03BC010F03AC00FF039C00EF070
:1048600019681868176816680DEC02F011C03CF062
:1048700010C03BF00FC03AF00EC039F001D140C07B
:1048800011F03FC010F03EC00FF03DC00EF0196AAD
:10489000186A176A0A0E166E0DEC02F011C040F08D
:1048A00010C03FF00FC03EF00EC03DF088510F0B1E
:1048B000216A206A1F6A1E6E3D261F503E2220502C
:1048C0003F2221504022A8D74D0E885DD8A442D067
:1048D000130E066E880E026EDEEC00F0D8A0D0D06B
:1048E000886F130E066E880E026EDEEC00F0D8A004
:1048F000C7D07C6E0D0E7C5C2DE1968988A19699BF
:104900009651E8B814D0D8909235E96EEA6AEA3642
:10491000E936EA36EC0EE926000EEA22EFCF2DF05A
:10492000ECCF2EF0ECCF2FF0ECCF30F013D0D890AE
:104930009135E96EEA6AEA36E936EA36980EE926F2
:10494000000EEA22EFCF2DF0ECCF2EF0ECCF2FF0BF
:10495000ECCF30F0470E885DD8A468D0130E066EF9
:10496000880E026EDEEC00F0D8A08AD0886F130E9D
:10497000066E880E026EDEEC00F0D8A081D07C6E50
:104980000D0E7C5CD8A452D0968D88A1969D965130
:10499000E8B814D0D8909235E96EEA6AEA36E9367A
:1049A000EA36EC0EE926000EEA22EFCF2DF0ECCF2E
:1049B0002EF0ECCF2FF0ECCF30F013D0D890913513
:1049C000E96EEA6AEA36E936EA36980EE926000E1A
:1049D000EA22EFCF2DF0ECCF2EF0ECCF2FF0ECCF82
:1049E00030F09651E8AC22D038C011F037C010F04A
:1049F00036C00FF035C00EF030C019F02FC018F0DF
:104A00002EC017F02DC016F0B9EC01F027C044F00D
:104A100026C043F025C042F024C041F04150355E2D
:104A20004250365A4350375A4450385A540E885DD3
:104A300027E1130E066E880E026EDEEC00F020E316
:104A4000886F130E066E880E026EDEEC00F018E31F
:104A50007C6E0D0E7C5C14E1978188A19791973153
:104A600008E3010EAA6E1F0EA96E010E80EC01F084
:104A700007D0010EAA6E1F0EA96E000E80EC01F089
:104A8000886B320E866FA6EC13F07EEC14F0BAEC55
:104A900011F0D4EC0BF0C0EF07F0800E016E0EECBD
:104AA00000F0080EF76EF60EF66E8DEC00F0800E3C
:104AB000016EC00E0EEC00F0090EF76E0C0EF66ED5
:104AC0008DEC00F0010E566E260E556E5504086EE4
:104AD000000E5658096E8A6B896B8951085C8A51A1
:104AE000095814E389515524A96E8A515620AA6E9B
:104AF00079EC01F0886F8AC0AAFF89C0A9FF8851AC
:104B000080EC01F0892B000E8A23E7E3886B99EF94
:104B100004F0000E415CE10E4258F50E4358050EBC
:104B2000445803E2200E0AEC01F0800E415C960E20
:104B30004258980E4358000E445803E2200E0AECE7
:104B400001F0040E016E056A44C011F043C010F07C
:104B500042C00FF041C00EF0196A0F0E186E420EDF
:104B6000176E400E166EB9EC01F011C021F010C0A6
:104B700020F00FC01FF00EC01EF05CEC00F02E0EF7
:104B80000AEC01F0030E056E44C011F043C010F0B2
:104B900042C00FF041C00EF0196A186A030E176E7A
:104BA000E80E166EB9EC01F011C021F010C020F033
:104BB0000FC01FF00EC01EF05CEC00F02E0E0AECD1
:104BC00001F0030E056E44C021F043C020F042C046
:104BD0001FF041C01EF05CEC00F0200E0AEC01F06A
:104BE000480E0AEC01F07A0E0AEC01F00D0E0AEC08
:104BF00001F00A0E0AEF01F0A1A41FD0A194010E4A
:104C0000AA6E0E0EA96E355080EC01F0365080EC85
:104C100001F0375080EC01F0385080EC01F0010ECB
:104C2000AA6E120EA96E915180EC01F0010EAA6ECF
:0E4C3000130EA96E925180EC01F0FFD7FFD752
:020000040030CA
:03000100C8191CFF
:02000500018177
:060008000FC00FE00F40E5
:0200000400F00A
:10000000013D1173016A5D1501A6C1EE01E64F3095
:10001000022F7045028CADA602EF91A80367EFFC9A
:1000200003ED7A37048A95500548D2FC0618F3711F
:10003000070821010812D08F092DA4570A61554ADB
:100040000C1C38D70DD71C631025A11E122A55424F
:1000500014C2AA95183871AE1B3F7FE41F23FFE03E
:1000600022E0A3B327A22E622B98CCA03070E35CD1
:10007000367EFFC83E47FFC048A9550A4F445CC5BD
:100080005731994060E1C6B86CFDFF907C8FFF80CE
:1000900048A9550A4F445CC55731994060E1C6B83C
:1000A0006CFDFF907C8FFF809152AA157F6F5F657A
:1000B000714B357F493F1D193D1725170F0D0B0F4C
:1000C0000B070F07090307050703030103010301DA
:1000D00001000100010000E0E0E0A060A0E00040BD
:1000E00040E0E000A02060A0A0A04060A000602050
:1000F000E02040006040E020A0006040E020A00040
:100100006040040506070009000B000000000044E1
:1001100095080C0200000000000200000000000131
:10012000FFFFFFFFFFFF013D1052016A5BCC01A6FC
:10013000C06E01E64D76022F6E49028CAB5502EF80
:100140008EFD0367ECE403ED76A6048A9130054842
:10015000CE2E0618EDE607081A9C0812C938092D9C
:100160009C000A614BDB0C1C2DD50DD70FCF102541
:100170009271122A44C014C297B618385BAA1B3F6A
:1001800067201F23E39222E08400272A0A5D2B9830
:10019000A5003070B755367ECE403E47C72448A9EB
:1001A00013004F4414BA57314A0060E16EAA6CFD47
:1001B0009C807C8F8E4948A913004F4414BA573154
:1001C0004A0060E16EAB6CFD9C807C8F8E49915241
:1001D00026007F6F5F65714B357F493F1D193D17C5
:1001E00025170F0D0B0F0B070F0709030705070353
:1001F00003010301030101000100010000E0E0E050
:10020000A060A0E0004040E0E000A02060A0A0A02E
:100210004060A0006020E02040006040E020A0009E
:100220006040E020A0006040040506070009000BC4
:1002300000000000004495080C02000000000002CD
:06024000000000000000B8
:00000001FF
